:020000020000FC
:10000000C4CDAEC10000000020C000008EC00000C2
:10001000000098C000000000000000000203040679
:10002000080C10182030406080000406080C1018DE
:100030002030406080A0C0000003070F1F000D0D9E
:1000400004050D050305030302004FB662FD0CC055
:10005000552041F00994C52DC095089483FDC7959E
:10006000C4BD64604FBE1895C0916400089483FDC0
:10007000C795C4BD6B7FC0916400CF3F09F41EC01B
:1000800070FF1AC082FD05C04FBE9198909893985A
:10009000189576FD0EC064FD0CC0C091B100C0FD86
:1000A0009498C1FD9798C2FD9598CAEFC095CA95DE
:1000B000F1F79198909893984FBE189524BCCC274F
:1000C000C064C8BF6460F8CFC6CF70FFC4CF64FD02
:1000D000C2CF919AC0CF70FFBECF64FDBCCF909AC3
:1000E000BACF70FFB8CF64FDB6CF939AB4CF949ACD
:1000F00070FFB1CF64FDAFCFC7E0CA95F1F7919A19
:10010000AACF979A70FFA7CF64FDA5CFC7E0CA9585
:10011000F1F7909AA0CF959A70FF9DCF64FD9BCF89
:10012000C7E0CA95F1F7939A96CF4FB6C9B7CF7E7D
:10013000C9BF6E7FCCB5CE0DDDB5DF1DDBBDCABD41
:100140004FBE18953FB68F7EABB7A074A2118061E9
:10015000A0E0ABBFA9B7AE7FA9BF7894A09168001B
:10016000AA2341F085FD2EC0A0916800AA95A09316
:10017000680028C040E050E085FD14C0A0B396FDA3
:10018000A095A2FD4FEFA3E096FDA2E0A5BFAA2790
:10019000A064AABF8D7FA0B396FDA095A2FD5FEFDE
:1001A000451741F7A8E161FDA093680085FD03C0F4
:1001B000A8E1A0936800409396008160442311F069
:1001C0002092990085FD0EC0A0916900AA2331F00C
:1001D000A0916900AA95A093690004C08061AA2734
:1001E000A064AABF80FF3CC0A09196004A2F61FF87
:1001F0008E7F85FD1CC0A091B400A430C1F4403FA7
:1002000008F040EFA42FA295AF704A0F5091B600AE
:10021000533069F0A695A69550FD01C0A69552FDF4
:1002200003C0A41B4A2F03C04A0F08F44FEF4093AA
:100230006100A72FA670A1F073FD12C0A0917000FD
:10024000AA0FAA0F50919E0056955695541708F084
:10025000452F4A0F4093610018F4AFEFA09361005F
:100260004091B400443009F03EC0A0916100A093D9
:10027000630040916300A0919B004A1708F04A2F49
:10028000A0919D004A1708F04A2F542EA091A0007B
:10029000AA2309F422C0542F5A1B10F4A42F50E0B3
:1002A000BA2E8894AA1FAA2EA091A200A095AA22D5
:1002B000A50E58F0A091A100A21509F0AA95AA0ECA
:1002C000A093A10048F04A2D08C0A091A100BA1641
:1002D00008F0A395A093A1004FEF409364007F7BAB
:1002E000485F08F07064A0916000A395A09360003F
:1002F00051F0F894A9B7A160A9BF84FF02C0A0E49F
:10030000ABBF3FBE1895A0917400A395A093740055
:1003100041E050916800552329F085FF03C05A95AC
:1003200050936800A0919600A13018F02092990097
:100330000DC020929A002092A300A0919900AF5F77
:10034000A093990018F0AFEFA0939900F894A9B783
:10035000A160A9BF84FF02C0A0E4ABBF3FBE189557
:100360003FB64CB55DB58F7EABB7A074A21180616E
:10037000A0E0ABBFA9B7AE7FA9BF789481FD23C031
:10038000A2E096FDA3E0A5BF8260A0B396FDA09574
:10039000A2FF05C040936500509366003EC1A3E0F4
:1003A00096FDA2E0A5BFAA27A064AABF8D7F85FF06
:1003B00001C026C140E0A0B396FDA095A2FD20C1DA
:1003C000409396000FC1A3E096FDA2E0A5BF8D7FEC
:1003D00061FF71C0A2E096FDA3E0A5BFAA27A064BB
:1003E000AABF82604093910050939200A0908F002A
:1003F0004A19B09090005B09BB24A22C4C385205DE
:1004000018F42092950049C0A091D400AA2359F174
:10041000483C520528F4A0E1BA2EAAE0AA2E23C037
:100420004836A1E05A0728F4A8E0BA2EAFE0AA2E79
:100430001AC0403DA2E05A0728F4A4E0BA2EAEE16B
:10044000AA2E11C0403AA5E05A0728F4A2E0BA2E1D
:10045000ACE3AA2E08C04839A8E05A0720F4A1E06E
:10046000BA2EA8E7AA2EC42EA0919300CA1AD52EA0
:10047000A0919400DA0ADD202AF4AFEFC094D09462
:10048000CA1ADA0A20929500A8E0A210A0E0CA14C5
:10049000DA0618F4A1E0A0939500409393005093DE
:1004A0009400409191005091920040938F0050939E
:1004B000900042E097C0A09165004A1BA0916600A1
:1004C0005A0B94FD82C093FD80C092FD7CC086FFD4
:1004D00003C0D52EC42E0CC05695479591FD73C010
:1004E0005695479590FD6FC0D52EC42ED694C794CF
:1004F00061FD19C0AC2DAC51AD2DA24008F005C076
:10050000DD2089F4AC2DA85C70F4A0916700A39560
:10051000AA2311F0A0936700AA3008F471C02092BA
:10052000960081606DC0A0916700AA2319F0AA957A
:10053000A0936700A22C5091BA0097FD06C0A0902E
:10054000C800533011F4A090D000AAEFAA0EA22D3B
:10055000A21DCA18DA0A4FB74170533049F4442338
:1005600021F087FD05C0806803C087FF01C08F7739
:10057000442359F0533031F4AFEFC094D094CA1AE9
:10058000DA0A03C040E050E020C0533049F4CC0CFC
:10059000DD1CAAE0CA1AD20818F4A0E0CA2ED22C98
:1005A000AFEFCA16D20418F04FEF50E00EC0A09182
:1005B000AC00CA9E412D000C441F50E008F012C050
:1005C0004FEF50E00FC05695479594FF07C0552355
:1005D00009F04FEFA42FA6954A0F521D4F3F520529
:1005E00008F04FEF40939600816061FF09C0AFE1D2
:1005F000A095A923AB299A2F8F7DBB2009F4806297
:10060000A8E1A093680085FF03C0AAE0A09368005A
:1006100061FD03C085FD01C08F7E85FD03C0A6E09E
:10062000A0936900F894A9B7A160A9BF84FF02C094
:10063000A0E4ABBF3FBE189511E00AC013E008C0AC
:100640001AE006C01EE104C014E602C018EC00C0A7
:1006500005E1BB27BA95F1F70A95D9F71A95C1F7C5
:1006600008952AE338E709C020E33CE806C02AE2FF
:1006700034EB03C025E238EC00C0B091AD00BA9570
:1006800009F4089512E0BB27979ABA95F1F7909A6A
:10069000BA95F1F79098BA95F1F79798BA95F1F75E
:1006A000123009F0919A123009F4939AB091AD008A
:1006B000BA95F1F7123009F09198123009F4939835
:1006C000B7E8BA95F1F71A95F1F6022FB22FBA955D
:1006D000F1F70A95D9F73A9581F6979A0895221B72
:1006E00039E0001F3A9509F40895221F211B18F4E0
:1006F000210F8894F6CF0894F4CF622C722CB0E0CE
:100700008894B395221F331FE0F737952795889477
:10071000912E802E020B130B10F4192D082D10F4BE
:10072000889401C00894661C771CBA9571F7172D40
:10073000062D0895322D11232AF43A95009510952F
:10074000031B130BF894029F712C002D129F912C08
:10075000802C7894780C172D921C292DB4E06B2EE8
:100760002695179507956A94D9F7332321F00095BC
:100770001095031B130B08950091B4000430A1F1F0
:10078000B0919600B15008F010C0B0916100B093E4
:10079000630020927E0020927F00209280002092B1
:1007A0008100209282006F7D1FC06090B400606263
:1007B000B0916100B093620008E317EC20917A00D9
:1007C00030917B0036952795B62DBA9541F0369538
:1007D0002795B62DBA95BA9511F0369527958DDFE8
:1007E00000937E0010937F00089500917E00B091E9
:1007F00062000B1B10917F00120928F40038BFEF34
:100800001B0740F009C00F37120508F405C00FE7B9
:1008100010E002C000E81FEF0093830010938400F3
:10082000089500918300B09180000B0F1091840017
:10083000B09181001B1F20E03091840033230AF423
:100840002A95B09182002B1F1AF4203F40F00AC075
:100850002F3008F407C00FEF1FEF2FE003C000E0B8
:1008600010E020EF30916300B0919B003B1718F42B
:10087000323030F009C0B0918400BB235AF004C07C
:10088000B0918400BB2332F4009380001093810068
:100890002093820008952091D70000918300000FDB
:1008A00010918400111F46DF11232AF40038BFEF96
:1008B0001B0740F009C00F37120508F405C00FE709
:1008C00010E002C000E81FEF002352F0B091620078
:1008D000B01B0B2F18F0013008F00AC001E008C06F
:1008E00000950F5FB09162000B0F08F001C00FEF91
:1008F0000093850008952091D80000918100109107
:10090000820018DF11232AF40130BFEF1B0740F0EB
:1009100009C00F3F120508F405C00FEF10E002C038
:1009200001E01FEF112352F0B0918500B01B0B2F97
:1009300018F0013008F00AC001E008C000950F5F10
:10094000B09185000B0F08F001C00FEF009363001A
:1009500008950FEF71FD1EC0B091D300BB23D1F0FD
:10096000B0917B00BB23B1F00FEF10917B00B7DE9D
:10097000F894B091730072FDB5E00B9F112D002D1E
:100980007894112309F00FEFB0919E000B1710F42B
:1009900000919E0000939D00089500917A001091AF
:1009A0007B0000541140B0919D0010F4BA9501C035
:1009B000B39511F0B0939D00089500C00895209163
:1009C000B500B6B1B6FDFBCF04B115B1B6B1BF7776
:1009D000B6B9B091AA00B395B093AA00B83060F14F
:1009E0002092AA00B091D200BB2321F1112329F05B
:1009F000B091AB00BF3F61F009C0B091AB000B17E5
:100A000039F020F4BB2321F0BA9502C0B395E1F38D
:100A100000919B00B093AB00B03050F400ECB030CC
:100A200038F400E8B03020F400E4B03008F400E01E
:100A300000939B007F7E089510919B00B0E11B0FF7
:100A400008F41FEF10939B00B091B400B43081F014
:100A500000919B00B0916300B01B10F40091630003
:100A6000B0919D000B1708F00B2F502E00936400DF
:100A7000B091AA00B73009F47061089502E3F894C8
:100A8000B091D9000B9F012D000C001F7894B091FC
:100A90009B000B1710F000919B00009361000093E6
:100AA0006300502E0093640000939E0008952092EE
:100AB0007A00B0EFB0937B000895F8940CB51DB5A3
:100AC00020917400789430917500609076000093C6
:100AD000750010937600031B160971FD03C077FDA6
:100AE00080C028C0709077002093770027092223C8
:100AF00019F00FEF1FEF0EC08090780090907900F2
:100B00003093780060927900009175001091760022
:100B10000819190920917A0030917B0036952795A4
:100B2000020F131F10F40FEF1FEF00937A001093C2
:100B30007B002BC020917A0030917B003901B4E01A
:100B40008B2EB2E09B2E343040F08A949A94383049
:100B500020F072FD02C08A949A94769467948A94E5
:100B6000E1F726193709992021F0169507959A94EF
:100B7000E1F7200F311F20937A0030937B0028F497
:100B80003FEF30937A0030937B00323008F4706886
:100B900071FF02C0B3E00DC0B091C40000917100BC
:100BA000023838F0B395003A08F0B395B63008F043
:100BB000B5E09B2EB4E08B2E10917B0000917A0063
:100BC00024E0169507952A95E1F70819120928F0EF
:100BD000B02FB250B12FB20910F402E010E098012A
:100BE00026C020917A0030917B0039017694679479
:100BF0006694669466942619320906950695200F28
:100C0000321D20937A0030937B00323008F07F77DA
:100C100004E0369527953695279526952695201B31
:100C200010F0223008F422E089019090C40060FDA9
:100C3000FECFE0908B00F0908C006160B9B7B0619E
:100C4000B9BF380177FD41C07694679400938B005B
:100C500010938C00B92DB330E1F0B0FD04C0060D47
:100C6000171D930106C0000F111F0250120922E048
:100C700030E0B92DB33068F020938D0030938E00B2
:100C800000938700109388006092890070928A0018
:100C90003AC000938D0010938E002093870030930C
:100CA00088006092890070928A0071FF0DC0BFE0D9
:100CB000B0938D0020928E00B093890020928A001C
:100CC000B0938B0020928C001EC0669400938B0022
:100CD000B92DB33091F0B0FD03C0060D262D03C031
:100CE000000F025022E0B92DB33038F020938D0070
:100CF000009387006092890006C000938D002093C6
:100D000087006092890000917C0002FD0350013051
:100D100031F495FD0CC0B2E0B06CB7B90BC0023035
:100D200021F4B3E0B06CB7B905C095FDF4CFB4E0E1
:100D3000B06CB7B90091A200000F10F4BBE60B270E
:100D40000093A20060FDFECFB2E0B0936E00616040
:100D5000B9B7B061B9BFB72FB670D1F020917A00A2
:100D600030917B00369527953695279571FF02C007
:100D7000B0E43B0FF8940CB51DB5020F131F1BBD5B
:100D80000ABD6160B0E1B8BFB9B7B061B9BF7894CE
:100D90000895686020927D0020E066FD20E206C094
:100DA000686020927D0020E266FD20E001E011E015
:100DB00077FD11C0B72FB67009F0677F14E100917D
:100DC0007B00069509F403950F3008F00FE071FFE2
:100DD00002C004E114E160FD0FC0B0917D00BB23AF
:100DE00059F071FF06C0B0916E00BA95B0936E00D5
:100DF00011F470624FC0ABDFB0B7B77FB0BFB8B10E
:100E0000B0B7B860B0BFB0917D00B395B0937D002E
:100E1000B8B177FD06C0B1E071FDB3E0BA95F1F766
:100E2000B8B1B072B21709F02AC071FF05C00395BE
:100E3000011708F00A95CFCF63FD05C00395011790
:100E400008F0B4CFC8CF677FF8943CB56DB470900C
:100E50007A00B0917B00770CBB1F08F4BFEF770CD2
:100E6000BB1F08F4BFEF370D6B1E6BBC3ABD616052
:100E7000B0E1B8BFB9B7B061B9BF789497CFB091BE
:100E80006D00B13008F492CF63FD90CF0A9509F060
:100E9000A2CF7F7D20918D0030918E00F894B0E13B
:100EA000B8BF0CB51DB5020F131F1BBD0ABDE090E6
:100EB0008700F09088006160B9B7B061B9BF7894DD
:100EC000B72FB67039F0B0916D0072FFB395B09343
:100ED0006D0009C075FF07C066FD05C063FD03C056
:100EE000BF91BF91FEC4089500E063FF01C001E01F
:100EF000F89410917100B7E01B9F212D102D78946C
:100F0000200F2695179526951795269517951093DA
:100F10007100183718F4B8E7B093710000917100B0
:100F2000B09172000B1720F060619198909893989F
:100F300060FDFECFE0908900F0908A006160B9B753
:100F4000B061B9BF0895B2E095FD0AC0F894B093BE
:100F50007C00979A949862FF01C0939A7894F4C0A9
:100F6000F894B0937C00979A959862FF01C0919A8B
:100F70007894EAC0B3E082FF24C095FD11C002E07E
:100F8000F894B0937C00E1E8F0E00093B10093980E
:100F9000959A62FF02C0909A01C097987894D4C045
:100FA00002E0F894B0937C00E1E8F0E00093B10037
:100FB0009198949A62FF02C0909A01C09798789491
:100FC000C3C095FD0BC0F894B0937C00EBE6F0E055
:100FD000939862FF01C0909A7894B6C0F894B09349
:100FE0007C00EBE6F0E0919862FF01C0909A789463
:100FF000ABC0B4E095FD0AC0F894B0937C00949A1D
:10100000959862FF01C0909A78949EC0F894B0932E
:101010007C00959A949862FF01C0909A789494C04D
:10102000B5E082FF24C095FD11C001E0F894B093B3
:101030007C00E7E7F0E00093B1009098979A62FF98
:1010400002C0919A01C0949878947EC004E0F8940C
:10105000B0937C00EBE8F0E00093B1009098979A91
:1010600062FF02C0939A01C0959878946DC095FD77
:101070000BC0F894B0937C00E5E6F0E0909862FF36
:1010800001C0919A789460C0F894B0937C00E1E735
:10109000F0E0909862FF01C0939A789455C0B6E052
:1010A00095FD0AC0F894B0937C00959A979862FFDA
:1010B00001C0919A789448C0F894B0937C00949AB7
:1010C000979862FF01C0939A78943EC0B1E082FF86
:1010D00024C095FD11C004E0F894B0937C00EBE8C7
:1010E000F0E00093B1009198949A62FF02C0939A45
:1010F00001C09598789428C001E0F894B0937C00E2
:10110000E7E7F0E00093B1009398959A62FF02C080
:10111000919A01C09498789417C095FD0BC0F894EB
:10112000B0937C00E1E7F0E0919862FF01C0939AF0
:1011300078940AC0F894B0937C00E5E6F0E09398C8
:1011400062FF01C0919A78946F7E089524E630E0A2
:10115000F9012092B100919890989398949A979A57
:10116000959A6B7F0895A2EBB0E009E00D9309E03A
:101170000D9304E00D930FEF0D9303E00D930FEF2C
:101180000D9309E00D9303E00D9301E00D9301E051
:101190000D93AEEBB0E001E00D930FEF0D930D93C7
:1011A0000D930D930D9303E00D930FEF0D930FEF40
:1011B0000D930D9305E20D9300ED0D9308E20D9351
:1011C00000E50D9304E00D930FEF0D9302E00D93F6
:1011D00000E00D930AE70D930FEF0D9300E00D93E0
:1011E00001E00D9300E00D9303E00D9300E00D93FB
:1011F00008952091B9008B7F233009F48460B09169
:10120000BA00B33019F09F7DB1FD90629F7BB09121
:10121000BB00B1FD9064223011F0886001C0877F6F
:1012200008950A95E00FF21DB4910895ECE1F0E005
:101230000091B200F6DFB093D700ECE1F0E000914E
:10124000B300EFDFB093D800EAE2F0E00091B8001D
:10125000E8DFB093D9000091B800023008F402E052
:1012600000937300B091CE000FEFB23009F400EAA2
:10127000B33009F402E800937200E8E3F0E0009173
:10128000D500CFDFB093A000089508952091C80045
:101290003091C900B091BA00B33009F43E5097FFC5
:1012A00002C020E03FEFB32FB21B6B2EB25810F4F8
:1012B000B2E86B2E00E00395609EB12DBD57D8F3C8
:1012C0000093AC0008959068E1DFBCD9BBD920E061
:1012D00030E0B0E16B2EB2D9B09196002B0F321DE9
:1012E0006A94C9F7B4E036952795BA95E1F7822E4E
:1012F0009F77CCDF0895F894E3E0F0E0B9E0B7BF62
:10130000B491B078C1F3F894A895B1B5B861B1BD06
:10131000B0E0B1BDB4E0BEBFBFE5BDBF17DFB0E018
:10132000B8BBB0E1B7BBB0E0B5BBB0E0B4BBB0EBAD
:10133000B2BBBBEBB1BB2224A0E0B0E02D92AA313E
:10134000E9F7A0E6B0E00FEF2D920A95E9F7B1E0DA
:10135000B093A20008DF01D3B7E0B06CB7B9B6B163
:10136000B460B068B6B90091CA000093AD00B1E0B6
:10137000B0936A00F8946AD974D964D975D962D9DE
:1013800076D960D9F8940AEF1AEFA0B396FDA0952C
:10139000A2FF1FC01A95C9F70A95B1F7E0E0FCE17A
:1013A000B591B43E39F4B591B03E21F4B591BF3F4B
:1013B00009F40CC0E0E0F395F395B591B83F49F41A
:1013C000B591B43931F4B591BA3A19F4EE27F695DE
:1013D00009940FDF2BDF59DF59DF0091CA0000931A
:1013E000AD00B4DEB2E0B3BFB2E0BEBDB2E0B5BDA9
:1013F000B1E5B8BFB9BFB0B7B77FB0BFB8B1B0B78C
:10140000B860B0BF19D97894D8DA20927000B3E0F0
:1014100096FDB2E0B5BFB0E4BBBFBB27B064BABFB6
:101420008D7F14D9626033E02CE0B0919500BB232E
:1014300021F42CE03A9509F4A5CF04D980FFA2CF7E
:101440008E7FB0919600B23078F3B92FBF710091C2
:10145000980000939700B0939800B01729F72A9549
:1014600021F76D7FB3E096FDB2E0B5BFBB27B06456
:10147000BABF8D7FB091D400BB2321F48062B92F15
:10148000B0709B2F8F7B20926700DED885FF05C050
:10149000B0916700BA3008F08064D0D802E085FFD0
:1014A00001C000E0B0919600B017B8F3F894D9D815
:1014B000D8D8D7D87894CAD820928600B091BA00EC
:1014C000B33009F47DC0BAD8B091BE00B13008F491
:1014D00077C0B0916A00B13008F472C085FD18C0C1
:1014E000B0919600BF3F08F46BC0F894C3D87894CD
:1014F000ABD8B0919600B130C0F7F894B2D8A0D86C
:10150000B0D87894A1D8B0919600BF3FB0F3E6C2AE
:10151000B3E09B2E9068F894B9DE789495D8F8944F
:101520009F77B4DE80909600B0919600BF37789494
:1015300008F44EC081D8F8949DD878949A9451F7C5
:10154000C2DEB82DB093C90081D8F8949AD27894AD
:10155000BAE09B2E9068F89499DE789475D8F89448
:101560009F7794DE80909600B0919600BF37789474
:1015700078F762D8F89475D863D873D878949A9429
:1015800049F7A1DEB82DBB5FB093C8000B2F1091B7
:10159000C900125810F0100B20F4B2E80B0F0093A2
:1015A000C90054D8F89406D27BD278944DD8F894D8
:1015B0006DDE7894B0919600BF3F08F48FCF8EC255
:1015C00000919600B09186000B1710F000938600F2
:1015D0003BD801E0B091BA00B35009F405E0B091F6
:1015E0009600B01708F06ACFF89444D843D842D890
:1015F00078942CD820926A0020926B0020926C0084
:10160000B0916B00B395B0936B00BF3F71F5B09193
:101610006C00B395B0936C00B091CC0009E1BA9521
:1016200059F002E3BA9541F00DE7BA9529F00AEFB7
:10163000BA9511F020926C00B0916C00B017A8F030
:1016400085DDFAD7B0916C00BA95B0936C0020920A
:101650006B00B091CB00B093AD00F8940BD87894A8
:10166000B091CA00B093AD00EFD7EAD7B09168004F
:10167000BB2319F485FF01C085CE01E085FD01C0C3
:1016800006E0B0919600B01708F4BACFB091BA0056
:10169000B35009F0D9D7B0916800BB2309F472CEDA
:1016A000F89454DD20926100209262002092630041
:1016B000522C209264002092A1007894B091B7003F
:1016C000BB0FB0939F0020927E0020927F0020925B
:1016D000800020928100209282002092AA0060E087
:1016E00070E020927100B8E0B093AA007061A4D7B6
:1016F000B7E074FDB7E0B06CB7B9B6B1B068B0642C
:10170000B6B9B6B1B6FDFDCF04B115B1B6B1BF776C
:10171000B6B9112309F00FEF0093AB0050D9B8E030
:10172000B093AA00706165DDF894BFEFB0939B00A1
:10173000A5D9B0916100B0939B00B0939C00B09389
:101740009D007894B1E0B0936100B09363005B2E8C
:10175000B0936400B093A400B0919A00B093A3003A
:10176000B091BA00B33019F49F7D87FD906271602B
:10177000726020926D0093DCA9DC99D99ED997D92B
:101780009CD995D90DDBF8D7AFDBDDDB96D901DB32
:1017900065FD2BD877FFDDD877FDFFD8A5DBEADB29
:1017A0008CD9FEDA65FD3DD89FDB23DC86D9F1DAE2
:1017B00065FD71D899DB34DC80D9F2DA65FD9BD800
:1017C00093DB6DDC7AD9E5DAB7E074FDB7E0B06C95
:1017D000B7B9B6B1B068B064B6B986DB77DC6DD99D
:1017E000EED871FF24C0B0919E00B0939B00B093DF
:1017F0009C00B0919A00B093A300B1E0B093A40014
:1018000018E12CE0B0916D00B11758F07D7F746045
:1018100020936F00B0919E00B0939B00B0939D0009
:1018200006C0B0919600B13008F0ACCF64C072FF32
:1018300015C066FD13C0B0916F00BA9519F47B7F97
:101840007860A0CFB0936F00B0919600B13008F0EF
:1018500099CFB091BA00B33009F04DC0209270001A
:10186000B09199000AEF1091D600112309F003E01E
:10187000B01708F040C085FF04C0B0916800BB23DA
:10188000D1F1B091BA00B33081F495FD03C087FD6A
:1018900004C00BC087FF01C008C066FD06C06064BD
:1018A000B0919E00B0939B0082CF00EF66FF05C011
:1018B000B0919E00B0939B0000E2B0917B00B01706
:1018C00008F460CF66FF17C06F7B9F7D87FD906235
:1018D0007460B2E1B0936F00B0919E00B0939B0032
:1018E00051CFB0917000B395B0937000B091960055
:1018F000BB2309F002C020927000F89427DC80908E
:10190000B900B2E0B093B90074DC8092B9002092C3
:1019100061002092620020926300522C20926400A9
:1019200020929F0060E070E078948ED60FDC0091EA
:10193000D600002319F0919A909A939AB7E0B06C70
:10194000B7B9B6B1B460B068B6B985FF05C0B0919B
:101950007000B43008F016CD4FCEEDE0F0E023D0AB
:10196000053509F01BC0EEE0F0E01DD00A3A09F0A1
:1019700015C03AE0A2EBB0E0E3E0F0E014D00D9344
:1019800031963A95D9F739E1AEEBB0E0EFE0F0E00F
:101990000AD00D9331963A95D9F702C0E4DB0AD00C
:1019A000E8E2F0E00895E199FECFEEBBFFBBE09ADC
:1019B0000DB308951ED03AE0A2EBB0E0E3E0F0E012
:1019C0000D910FD031963A95D9F739E1AEEBB0E0F1
:1019D000EFE0F0E00D9105D031963A95D9F712D0AD
:1019E0000895E199FECF0DBBEEBBFFBBE29AE19AF1
:1019F0000895EDE0F0E00FEFF4DFEEE0F0E00FEF40
:101A0000F0DF0895EDE0F0E005E5EBDFEEE0F0E07B
:101A10000AEAE7DF08953091AE000091AF0031305F
:101A200011F40093B200323011F40093B30033305C
:101A300011F40093B400343011F40093B600353043
:101A400011F40093B800363011F40093C40037301D
:101A500011F40093B900383011F40093D5003930F7
:101A600011F40093CE003A3011F40093BA003B30E9
:101A700011F40093BB00089525E0E8D52A95E9F715
:101A80000895EFD5F1D5F3D5F5D5DAD5EAD5ECD56E
:101A9000EED5F0D5D5D5E5D5E7D5E9D5EBD5089583
:101AA000E9D5E5D5E1D5DDD5CBD5E4D5E0D5DCD597
:101AB000D8D5C6D5DFD5DBD5D7D5D3D50895809079
:101AC000AE009090AF00CDD5CCD5CBD5B9D58A940A
:101AD000D1F7D0D5B5D59A94E1F70895F894D1DF30
:101AE0007894CADFC9DFB1E0B093AE00B1E0B09343
:101AF000AF002092B000F894E2DF7894B5E06B2E4E
:101B000070909600A3D5B09196007B16C9F7B130BE
:101B100018F0BF3F40F107C07EDFF8944BDFB1DF24
:101B2000B8E0B1BDA9DF6A9459F7B091B000B395A0
:101B3000B093B000B33008F4DECF9EDFB091AF00B9
:101B4000B395B093AF00F894B091AE00BA95EEE3C0
:101B5000F0E0EB0FF21D049178940395B091AF0083
:101B6000B01708F4C6CF88DF87DFB091AE00B39519
:101B7000B093AE00B091AE00BC3008F4B7CFF3DA4A
:0C1B8000F89418DFB8E0B1BD77DFB5CBFA
:00000001FF
